:1000000038C055C14FC04EC04DC04CC04BC04AC097
:1000100049C048C047C046C045C044C043C042C0B4
:1000200041C040C03FC00403090412036F006200D6
:100030006400650076002E00610074001203540015
:1000400065006D0070006C006100740065001201B5
:100050001001FF000008C016DC05000101020001CC
:1000600009021200010100801909040000000000CB
:10007000000011241FBECFEDCDBF10E0A0E6B0E020
:10008000E8E5F5E002C005900D92A236B107D9F778
:1000900010E0A2E6B0E001C01D92AD38B107E1F773
:1000A00033D258C2ADCF1F93CF93DF9380917300AB
:1000B000835087FD7EC09091700020916F002D329B
:1000C00009F075C0883009F072C0CCE0D0E0C91BDF
:1000D000D109C958DF4F83EC809363008AE5809390
:1000E0006000109262008881807619F0CE0127D2DC
:1000F00055C09A8110926C008981882331F4109246
:100100006D002CE630E082E045C0853019F4909314
:10011000740036C0863059F58B81813019F48EE435
:1001200090E01AC0823019F480E690E015C0833068
:10013000C9F4992341F486E290E090937200809391
:10014000710084E010C0913019F48AE290E004C09C
:10015000923041F48CE390E09093720080937100B0
:1001600082E101C080E090E49093620017C0883083
:1001700059F0893019F49093760002C08A3039F032
:100180002CE630E080E006C026E730E002C02CE636
:1001900030E081E030937200209371009F819923B9
:1001A00021F49E81981708F4892F809361001092A2
:1001B00073008091600084FF4CC0809161008F3F8C
:1001C00009F447C0182F893008F018E0811B80938C
:1001D00061008091630098E8892780936300112370
:1001E00061F1809171009091720030916200212F35
:1001F000215036FF0EC030E0A9014B595F4FFC0182
:10020000A4E6B0E064916D933196A417B507D1F7D9
:100210000CC0DC0130E0A9014B595F4FE4E6F0E08F
:100220006D916193E417F507D9F72F5F3F4F280FC2
:10023000391F309372002093710084E690E0612FA3
:1002400032D01C5F1C3019F08FEF80936100109347
:10025000600084E190B39C7031F48150D9F7109222
:10026000740010926E00DF91CF911F91089585B7B1
:10027000826085BF8BB780648BBF0895A82FB92F8C
:1002800080E090E041E050EA609530E009C02D91B7
:1002900082279795879510F084279527305EC8F3BD
:1002A0006F5FA8F30895EADF8D939D930895CF9330
:1002B000CFB7CF93C395839BE9F7839B09C0839BFB
:1002C00007C0839B05C0839B03C0839B01C0A1C063
:1002D000DF93C0917000DD27C958DF4F839B02C0B8
:1002E000DF91EBCF2F930F931F9300B32FEF03FBFF
:1002F00020F94F933F9310B34FEF012703FB21F9F0
:100300003BE031C04E7F012F10B3216028C0102F79
:100310004D7F2260000000B329C04B7F2460012F75
:10032000000010B32BC010B3477F28602AC04F7E57
:1003300000B320612CC04F7D10B320622FC04F7BD3
:1003400000B3206432C0422700B349934FEF00004E
:10035000102713FB20F910B31C70C9F1297F91F20B
:10036000012703FB21F900B3237F89F2315058F1B3
:10037000102713FB22F910B3277E79F2012703FB24
:1003800023F92F7C81F200B3102713FB24F92F7976
:1003900071F200C010B3012703FB25F92F7359F246
:1003A00000C000B3102713FB26F9223040F200C032
:1003B00010B3012703FB27F9243028F64F77206874
:1003C00010B30000F9CF10E41ABF002717C03B504C
:1003D0003195C31BD04010E41ABF0881033CE9F0FB
:1003E0000B34D9F020916E001981110F1213EDCF4B
:1003F000093641F10D3211F0013E39F700937500D5
:100400003F914F911F910F912F91DF91CAB7C6FD78
:1004100051CFCF91CFBFCF91189520917500222356
:1004200079F310917300112311F5343012F13093E8
:10043000730020936F00109170003BE0311B3093EC
:10044000700017C00091730001308CF40AE5309100
:10045000600034FD10C000936000C3E6D0E00FC020
:100460002795A8F45150A9F4220F0000F9CF4AE5CE
:1004700003C042ED01C0432FC4E1D0E032E011B32C
:100480001C60939A11BB02B320E41CE05F93012728
:1004900056E002BB279520F4515021F4220FF9CFEA
:1004A000012756E000003B5A02BBD0F2279528F402
:1004B000515029F4220F0000F9CF012756E027956B
:1004C00002BB20F4515021F4220FF9CF012756E04E
:1004D0002991332302BB21F6037F10917400110F81
:1004E000C651D04002BB11F010936E0010E41ABF49
:1004F000086011B3137F402F437F5F9100C000C09D
:1005000002BB11BB42BB7CCF8E9A2EE088E190E00B
:100510000FB6F894A89581BD0FBE21BDA8DE8B9AB9
:100520008AEFA895EFE6F7E13197F1F700C00000F8
:100530008150B9F78B987894A895B5DDFDCFFC0173
:100540008181882321F0813019F4969A01C0969810
:0805500080E00895F894FFCF4C
:020558005AFF48
:00000001FF
